:020000040000FA
:100000008316FF308500FF2390009F01053081009B
:100010009516151696168312073099008B15203009
:100020008400DF008001840ADF08031D1228952068
:10003000B33081000B110A30B0007E20031D22284E
:10004000A50A1D281121A600250203182A2803014C
:10005000A600022126082406031930287E202A281B
:100060006020A2200030051EFF308500C100411233
:100070008316F830850083123D28C00F43284108BD
:1000800085000B191721C108031D532840083707A5
:100090000318051540083507031885144008330771
:1000A000031805143D2840083707031805114008B8
:1000B00035070318851040083307031805103D283D
:1000C0007A20A700013E0319752827308400840A8E
:1000D000A20A0319A30A7A2080002B300406031D0C
:1000E0006728A20A0319A30A08002008A200210811
:1000F000A300602823088A00220882009E20013E77
:10010000031987280530A0070318A10A7E28A40A2E
:10011000A00A0319A10A9E20013E03199528200870
:10012000A2002108A30003010800A4010130A100DE
:10013000A3007930A000A200FF38080021088A003F
:10014000200882002808B1002708AF00031DB0284E
:100150002908B3002A08B5002B08B700BF01080022
:100160000730BF000130B200B400B60033082902E6
:100170000318BD28B203B203003CB80035082A02B8
:100180000318C528B403B403003CB90037082B0298
:100190000318CD28B603B603003CBA00380839026C
:1001A0000318D92838083A023A080318DE28380814
:1001B000DE2839083A023A08031C3908003CBE0020
:1001C000BB00BC00BD0008002408022141088500D6
:1001D000831605128312851EEB280F30FA200508BE
:1001E0000B10630000005A30FA20851AEB28851E98
:1001F000F728002881010B110B1DFC28FF3E031D71
:10020000FA2808008512831685129A009B018C1328
:100210001C1555309D00AA309D009C148516831234
:10022000080083169B011C141A0883120800010899
:10023000B33E81000B11AE0803192429AD0B24290C
:10024000AE0B242924080221851A2A29AC0A031995
:10025000E4283B29FC302C0703183029AC013B294A
:100260007E206020B301B501B701A2200A30B000A2
:10027000AC010830AE00BF0803196D29AF0B0800B0
:100280002708AF0029083306031D48293F105029CD
:100290003808BB07031C50293E08BB073208B307C8
:1002A0002A083506031D5629BF105E293908BC07E8
:1002B000031C5E293E08BC073408B5072B08370627
:1002C000031D64293F1108003A08BD07031C0800FC
:1002D0003E08BD073608B7070800B108031976299C
:1002E000B00B08000A30B000B10B08006020A2205B
:1002F000080000340534FF34003400340134003485
:10030000003400340034003405340034FF34003449
:100310000134003400340034003400340534003437
:100320000034FF3401340034003400340034FF342E
:1003300002340134FF340034003402340134003418
:10034000FF3400340234013400340034FF34FF340D
:1003500002340134FF344034003402340134403478
:100360000034FF34023401340034FF344034FF34AD
:100370000034FE34FF3400340034FF340034FE34E3
:100380000034FF340034FF340034FE3400340034D1
:10039000FF34FF340034FE34F0340034F034FF34E2
:1003A0000034FE34FF349B340034FF340034FE3418
:1003B000F034F034F034FF340034FE3480348034D0
:1003C0008034FF340034FE34303430343A34FF3477
:1003D00000340134FF34003400340034013400347C
:1003E000FF3400340034013400340034FF34FF346F
:1003F0000334003480348034803400340134C83411
:10040000FF34FF340034013400340034003400344D
:100410000134C834FF34FF34003401340034003474
:10042000003400340134C834FF34FF340034013464
:1004300000340034003400340134C834FF34FF3455
:100440000034013400340034003400340134C83442
:10045000FF34FF34003401340034003400340034FD
:100460000134C834FF34FF34003401348034803424
:10047000803402340234003400340034FF34063453
:100480000A34FF340034003406340A34FF34FF34B5
:10049000003406340A340034FF34003406340A349D
:1004A0000034FF34FF3406340A3400340034FF349F
:1004B00006340A34FF340034FF34FF341934FE3478
:1004C000FF34003400341934FE34FF34FF34003478
:1004D0001934FE340034FF3400341934FE3400344F
:1004E000FF34FF341934FE3400340034FF3419343F
:1004F000FE34FF340034FF34FF3404340A34FE3455
:100500002034003404340A34FE348034003404349B
:100510000A34FE34F034003404340A348034F034C5
:100520000034FF3404340A3400341034FF3404340B
:100530000A3400348034FF3404340A340034F03494
:10054000803404340A3410341034F03404340A345F
:10055000F0341034F03404340A3440340034FA34C3
:10056000FF340A340434F0340034F0340A340434F0
:1005700020340034F0340A340434803400348034BD
:100580000A340434F03400342034FF3400340534A9
:10059000003400340A3400340534003400340034AC
:1005A000FF34FF34723467346234733461345F343F
:1005B00069346E34653474342E34613473346D347C
:1005C0002034303439342F34303436342F3432340C
:1005D0003034303437342034523432342E343034E2
:1005E0002E34323428346334293420345034653482
:1005F0007434653420344734723469346634663474
:1006000069347434683473342034323430343034E0
:1006100036342D343234303430343734203472347C
:100620006734623473346134403470346534743404
:100630006534733477346F3472346C3464342E34EC
:10064000643465346D346F346E342E3463346F34F7
:060650002E3475346B34FA
:02400E00A43FCD
:00000001FF
